:04000000DFEF08F036
:1000080000C016F001C015F0E1CF17F0E2CF18F0EC
:100018009DAA69D09EAA67D0AECFC9F0ABA20FD077
:10002800AB98AECFC9F0AB88010E0201D625006EA1
:10003800000ED721016E00C0D6F201C0D7F2ABA4E2
:100048000FD00201AB9EAB8E010ED625006E000EBE
:10005800D721016E00C0D6F201C0D7F2AECFC9F0E9
:100068000001C9510D0A08E00201D951000802E156
:10007800D8517E0801E320D00201010E446F000E22
:10008800456FD951000802E1D8517E0804E2020EFA
:10009800446F000E456F9D9A460ED825E16E020EFC
:1000A800D921E26EE66AD8C2D4F2D9C2D5F2D86BA9
:1000B800D96B0001C96B17D0460E0201D825E16E35
:1000C800020ED921E26EC9C0E6FFD8C2D4F2D9C265
:1000D800D5F2010ED825006E000ED921016E00C0A0
:1000E800D8F201C0D9F29DA01DD09EA01BD0010E50
:1000F8003F5C006E000E4058016E00C03FF001C02A
:1001080040F0000E405C02E1010E3F5C06E29D906B
:10011800CD90010E3D6E000E3E6E3C0ECF6EB00EC1
:10012800CE6E9E9016C000F015C001F017C0E1FF1A
:0601380018C0E2FF1100F7
:10013E0000C304F08B94060E0D6E0D2EFED700003C
:10014E00026A036A800E0318006E800E005C02E1E4
:10015E00080E025C1CE2800E0414016E0150800A2F
:10016E0002E18B8401D08B940D0E0D6E0D2EFED7F9
:10017E00043604908B800D0E0D6E0D2EFED78B90D7
:10018E000D0E0D6E0D2EFED7024A032ADBD712007E
:10019E00FAC201F3FBC202F30301013701910237E8
:1001AE00080E036F000E046F0201FE6BFF6B800ED4
:1001BE00FF19006E800E03010419005C03E1035168
:1001CE000201FE5D0BE20201380EFE25E16E010E0C
:1001DE00FF21E26EE66AFE4BFF2BE9D7010E03010B
:1001EE000125006E000E0221016E380E0024E16E14
:1001FE00010E0120E26EFCC2E6FF380E0125E16E13
:10020E00010E0221E26EFDC2E6FF8B9203C3FEF2E7
:10021E0004C3FFF2800E006E800E0201FF19005C17
:10022E0002E1FE51000815E2010EFE5D006E000EA9
:10023E00FF59016E380E0024E96E010E0120EA6EA0
:10024E00EECF00F375DF010E0201FE5F000EFF5BC5
:06025E00E1D78B821200C3
:10026400800E0201F419006E800E005C02E1000EA3
:10027400F35D0BE3800EF419006E800E000A005C3F
:1002840002E1040EF35D01E201D047D0800EF619BD
:10029400006E800E005C02E1000EF55D0AE3800E44
:1002A400006E800EF619005C02E1F551080801E3C6
:1002B40001D033D0030E026EF3C200F0F4C201F099
:1002C400025005E0003600900136FF0FFAD700C057
:1002D400F8F201C0F9F2F5510026F6510122410E5F
:1002E4000024E16E000E0120E26EF7C2E6FFF3C2C5
:1002F400FAF2F4C2FBF2F551010FFC6FF551F82547
:10030400006EF651F921016E410E0024E96E000ED3
:0C0314000120EA6EEECFFDF240DF120087
:10032000220E0C6E086A096A0A6A0B6A0C06D8B4B7
:100330001FD0D8900B320A3209320832033202320F
:1003400001320032D8A0F2D70C06D8B409D004503C
:1003500008260550092206500A2207500B22EAD728
:10036000045008260550092206500A2207500B2285
:02037000120079
:100372000B6A0C6A800E0C18006E800E005C02E1A3
:10038200080E0B5CD8B0A0D00BC003F00CC004F078
:1003920003360390043603C000F004C001F00036B7
:1003A20000900136003600900136F80E0024096EE6
:1003B200010E01200A6E09C0E9FF0AC0EAFFEECF72
:1003C20005F0EECF06F0EECF07F0EECF08F01F0EED
:1003D200046E05C000F006C001F007C002F008C0BC
:1003E20003F0045007E00332023201320032039E6E
:1003F200FF0FF8D700C00DF005C000F006C001F0F5
:1004020007C002F008C003F0003600900136023641
:10041200033609C0E1FF0AC0E2FF00C0E6FF01C0E7
:10042200E6FF02C0E6FF03C0E6FF0BC000F00CC00F
:1004320001F0003600900136010E0024036E000E1A
:100442000120046E03C000F004C001F000360090E9
:100452000136003600900136F80E0024096E010EB6
:1004620001200A6E09C0E9FF0AC0EAFFEECF05F0DB
:10047200EECF06F0EECF07F0EECF08F005C000F0A9
:1004820006C001F007C002F008C003F00036009079
:100492000136023603360D500012000E011202120E
:1004A200031209C0E1FF0AC0E2FF09C0E1FF0AC06E
:1004B200E2FF00C0E6FF01C0E6FF02C0E6FF03C0A4
:0A04C200E6FF0B4A0C2A56D7120081
:1004CC008B92130E0D6E0D2EFED700000000EDC2A8
:1004DC0000F32FDEF1C200F32CDEEDC200F329DEB7
:1004EC00F0C200F326DEEDC200F323DEEFC200F310
:1004FC0020DEEDC200F31DDEEEC200F31ADE0D0E9F
:0A050C000D6E0D2EFED78B8212003B
:10051600A00E0201EF6F0F0EF06F000EF16FF26F7B
:10052600A00E006E0F0E016E000E026E000E036E20
:10053600EDC204F0EEC205F0000E066E076EEDDEAB
:1005460000C0EFF201C0F0F202C0F1F203C0F2F215
:10055600000E035C08E1000E025C05E1020E015C80
:1005660002E1940E005C01E231D0940EEF5F020EC0
:10057600F05B000EF15BF25B050E006E005007E0CB
:10058600F233F133F033EF33F29FFF0FF8D7EFC2B8
:1005960000F0F0C201F0F1C202F0F2C203F0010E67
:1005A600EF5F000EF05BF15BF25B00500110021092
:1005B60003100CE000000000000000000000000036
:0E05C60000000000000000000000E1D712005D
:1005D4000201F16BF26B800EF219006E800E005C6A
:1005E40002E1080EF15DD8B094D0F1C200F0F2C27D
:1005F40001F0003600900136010E0024036E000E57
:100604000120046E03C000F004C001F00036009025
:100614000136003600900136F80E0024E96E010E12
:100624000120EA6EEECF00F0EECF01F0EECF02F043
:10063400EECF03F000C0EDF201C0EEF202C0EFF223
:1006440003C0F0F2FF0E0014F76FF36BF46BF1C20A
:10065400F5F2F2C2F6F204DEF1C203F0F2C204F0E3
:1006640003360390043603C000F004C001F00036E2
:1006740000900136003600900136F80E0024E96E31
:10068400010E0120EA6EEECF05F0EECF06F0EECFBC
:1006940007F0EECF08F005C0EDF206C0EEF207C099
:1006A400EFF208C0F0F208C000F0016A026A036ABF
:1006B400010EF36F000EF46FF1C2F5F2F2C2F6F21E
:1006C40000C0F7F2CDDDEFC200F0F0C201F0026A23
:1006D400036A020EF36F000EF46FF1C2F5F2F2C278
:1006E400F6F200C0F7F2BCDDEEC200F0EFC201F09A
:1006F400F0C202F0036A030EF36F000EF46FF1C24E
:10070400F5F2F2C2F6F200C0F7F2AADDF14BF22BD9
:0407140062D7120096
:0E071800670E0D6E0D2EFED7000000001200C1
:0A07260000000000000000001200B7
:0E073000ACB202D00000FCD7E8C2ADFF120050
:10073E00030E0C6E950E0D6E0D2EFED70C2EFCD7E5
:02074E00120097
:100750000201E86BE96B800EE919006E800E005C07
:1007600002E1080EE85D11E2E851010FED6FEE6B5A
:10077000EF6BF06BF16BAADE1A0E0D6E0D2EFED72D
:0C07800000000201E84BE92BE6D7120054
:10078C00800E0201E919006E800E005C02E1200E61
:10079C00E85D0AE3800E006E800EE919005C02E150
:1007AC00E8517F0801E307D0000EE91902E1860E3B
:1007BC00E81901E070D0EA6BEB6B000EEB5D02E127
:1007CC00080EEA5D5BE2200EE85D036E000EE9594F
:1007DC00046E030E026E03C000F004C001F0025060
:1007EC0005E0003600900136FF0FFAD7EA510026DB
:1007FC00EB510122D80E0024F66E160E0120F76E76
:10080C00000EF86E000EF8220900F5CF06F0EAC2D1
:10081C0003F0EBC204F003360390043603C000F07F
:10082C0004C001F00036009001360036009001360D
:10083C00F80E0024046E010E0120056E04C0E9FFC1
:10084C0005C0EAFF0650EE10006EEECF01F0EECFC1
:10085C0002F0EECF03F0000E01120212031204C0DC
:10086C00E1FF05C0E2FF00C0E6FF01C0E6FF02C0E9
:10087C00E6FF03C0E6FFEA4BEB2B9FD7EC6B080EB1
:10088C00EC5D09E270DDA0DE3BC0EDF23CC0EEF2A7
:08089C003CDEEC2BF4D7120046
:0C08A400420E0D6E0D2EFED7000012005B
:1008B000086A096A100E0C6E0134083609360450B5
:1008C000085E0550D8A0053C095ED8B007D004509A
:1008D00008260550D8B0053C0926D89000360136C8
:0608E0000C2EEAD7120005
:1008E600086A080E0C6E003408360450085ED8B04C
:0E08F60002D00826D89000360C2EF5D712003E
:100904000B6A0A6A096A00500402F4CF09F0F3CFB3
:1009140008F001500502F4CF0BF0F3CF0AF00050B9
:100924000502F3500926F4500A22E86A0B2201500A
:100934000402F3500926F4500A22E86A0B2208C084
:1009440000F009C001F00AC002F00BC003F012006D
:10095400DEC204F0DFC205F004C0E9FF05C0EAFF0F
:10096400EE5203E0044A052AF7D704C002F005C09A
:1009740003F0044A052AE0C200F0E1C201F00201DA
:10098400E04BE12B00C0E9FF01C0EAFF02C0E1FF38
:1009940003C0E2FFEECFE6FF02C0E9FF03C0EAFFB7
:1009A400EE5201E0E2D7DEC200F0DFC201F0120035
:1009B4008B92030E0B6E080E0C6E770E0D6E0D2EC1
:1009C400FED70C2EFCD70B2EFAD70F0E0201ED6FBB
:1009D400EE6BEF6BF06BF16B77DD090E0201ED6FDF
:1009E400EE6BEF6BF06BF16B6FDD0A0E0201ED6FD6
:1009F400EE6BEF6BF06BF16B67DD0B0E0201ED6FCD
:100A0400070EEE6F070EEF6F070EF06F070EF16F14
:100A14005BDD0C0E0201ED6F010EEE6F010EEF6F48
:100A2400010EF06F010EF16F4FDD0B0E0C6E620EB6
:100A34000D6E0D2EFED70C2EFCD7000087DE340E73
:100A44000C6EF10E0D6E0D2EFED70C2EFCD7000091
:040A5400000012008C
:100A5800E0C201F0010E006E015004E00036009083
:100A6800FF0FFBD700C0E2F2001EDEC2E9FFDFC2C3
:100A7800EAFF0050EF16120EE9260050EF165BDE73
:100A88000201E251EF12120EE95E42DEE251EF146A
:100A9800E16FE151000A000ED8A4010EE16F4BDEB0
:060AA800E1C200F01200A3
:100AAE00020E0C6E4B0E0D6E0D2EFED70C2EFCD7BD
:020ABE00120024
:100AC0000900F5CFE6FF0006FBE10106F9E112009F
:100AD000300E0201C66F070EC76FE80EC86F020E18
:100AE000C96FFF0E386FFF0E396F000E3A6F000EA0
:100AF0003B6FFF0E3C6FFF0E3D6F000E3E6F000E12
:100B00003F6FFF0E406FFF0E416F000E426F000EF1
:100B1000436FAC8A900EAB6E948E949C9EAA03D0C9
:080B2000AECF00F0FBD712007C
:100B2800E0C201F0010E006E015004E000360090B2
:100B3800FF0FFBD700C0E4F2001E00C0E3F2DEC2E4
:100B4800E9FFDFC2EAFF0050EF16120EE9260201A4
:100B5800E26BE251070815E3E2C200F0E1C201F0DE
:100B6800005004E00132019EFF0FFBD7E351EF165E
:100B780001A002D0E451EF12CBDDE451EF12E22BD9
:0C0B8800E8D7120EE95E8ADE89DE12005A
:100B9400030E0B6E080E0C6E770E0D6E0D2EFED727
:0A0BA4000C2EFCD70B2EFAD712001E
:100BAE00DEC2F6FFDFC2F7FFE0C2F8FF0900F5CFA5
:100BBE0000F0005211E0DEC2F6FFDFC2F7FFE0C226
:100BCE00F8FF0900F5CFE8F2ACDD010E0201DE27D9
:100BDE00000EDF23E023E4D7060E0D6E0D2EFED79A
:040BEE0000001200F1
:100BF2000201E06BE16B800EE119006E800E005C79
:100C020002E1400EE05D0AE2890EE025E16E000E8F
:100C1200E121E26EE66AE04BE12BEDD7E26BE36B9A
:100C2200DEC2E9FFDFC2EAFFEE500008D8B08BD087
:100C3200DEC2E9FFDFC2EAFF200EEE5CE46F030EC4
:100C4200006E000EE56F005005E0E437E491E537F1
:100C5200FF0FFAD7E06BE16B800EE119006E800E98
:100C6200005C02E1080EE05D67E2E051E225006E01
:100C7200E151E321016E890E0024E16E000E012094
:100C8200E26EE051E425006EE151E521016ED80EDD
:100C92000024F66E160E0120F76E000EF86E000E9E
:100CA20001BEFF0EF8220900F5CF00F000C0E6FFFA
:100CB200E051010FED6F890EE025E96E000EE12192
:100CC200EA6EEECFEEF2080EE025006E000EE12194
:100CD200016E890E0024E96E000E0120EA6EEECF4D
:100CE200EFF2100EE025006E000EE121016E890E7A
:100CF2000024E96E000E0120EA6EEECFF0F2180E2B
:100D0200E025006E000EE121016E890E0024E96EDD
:100D1200000E0120EA6EEECFF1F266EC02F0060E52
:100D22000C6E300E0D6E0D2EFED70C2EFCD7000071
:100D32000201E04BE12B90D7080EE227000EE323DD
:080D4200DE4BDF2B6DD7120020
:100D4A000D0E0201E86FEFDC0A0E0201E86FEBDC20
:020D5A00120085
:100D5C000201E56BDFAF0DD0010EE56FE0C2E1FFE4
:100D6C00E1C2E2FF2D0EE66EDE1FDF1FDE4BDF2B36
:100D7C0007D0E56BE0C2E1FFE1C2E2FF200EE66EB8
:100D8C00DEC200F0DFC201F001320032019E0132FE
:100D9C000032019E01320032019E01320032019E6E
:100DAC0000C0E2F2010EE025E66F000EE121E76FD4
:100DBC000A0E046E92DD0A0E046E8FDD08C000F080
:100DCC00300E0026E6C2E1FFE7C2E2FF00C0E6FFFC
:100DDC00010EE025E96E000EE121EA6EEE50300ABC
:100DEC0008E1010EE025E16E000EE121E26E200E1D
:100DFC00E66E020EE025E66F000EE121E76F0A0EAB
:100E0C00046EE2C200F069DD08C000F0300E00266E
:100E1C00E6C2E1FFE7C2E2FF00C0E6FFDEC2E3F29A
:100E2C00DFC2E4F20F0EDE15006EDFC201F0000E21
:100E3C00011600C0E3F201C0E4F2710E046E020E62
:100E4C00056E5ADD00C0E3F201C0E4F2030EE025AA
:100E5C00E16E000EE121E26E2E0EE66E040EE02530
:100E6C00E66F000EE121E76FE80E046E030E056ECF
:100E7C00E3C200F0E4C201F015DD300E0026E6C23C
:100E8C00E1FFE7C2E2FF00C0E6FF050EE025E66FDA
:100E9C00000EE121E76F640E046E000E056EE3C2D6
:100EAC0000F0E4C201F0FEDC0A0E046E000E056ECA
:100EBC00F9DC08C000F009C001F0300E0026E6C2D3
:100ECC00E1FFE7C2E2FF00C0E6FF060EE025E16E9F
:100EDC00000EE121E26EE66A070EE025E16E000EDF
:100EEC00E121E26EE66A080EE025E16E000EE121DA
:100EFC00E26EE66AE551010A13E1E2C200F0000E6F
:100F0C00016EE80E046E030E056EF6DCE351002450
:100F1C00376EE4510120386E000E396E3A6E17D0E0
:100F2C00E2C200F0000E016EE80E046E030E056EB8
:100F3C00E3DCE3510026E451012200500008376E37
:100F4C0001C038F0000E3856000E396E3A6E1200A1
:100F5C00310ECD6E3C0ECF6EB00ECE6EDEC23FF0BB
:100F6C00DFC240F03D6A3E6ACD809E909D801200AB
:100F7C000201E06BE16BE26BE36BE051DE25E96EA5
:100F8C00E151DF21EA6EEECFE2F2000EE36F000ECC
:100F9C00E36F000EE31902E1000EE21910E0000EFF
:100FAC00E31902E1270EE21904E1860EE26F000E4E
:100FBC00E36FE2C2E8F2E3C2E9F2C6EC03F0E04B05
:100FCC00E12B000EE31902E1000EE219D6E112004A
:100FDC00E0C2F6FFE1C2F7FFE2C2F8FF0900F5CF6D
:100FEC0000F0005218E0E0C2F6FFE1C2F7FFE2C2E7
:100FFC00F8FF0900F5CF00F0DEC2E1FFDFC2E2FF2F
:10100C0000C0E6FF0201DE4BDF2B010EE027000ED5
:10101C00E123E223DDD7DEC2E1FFDFC2E2FFE66AB5
:02102C001200B0
:10102E00310ECD6ECD823C0ECF6EB00ECE6E9E903A
:10103E009F803F6A406A3D6A3E6ACD909D90120045
:10104E00E0C201F0010E006E015004E00036009087
:10105E00FF0FFBD700C0E4F2001C0201E36FE26B4E
:10106E00DEC2E9FFDFC2EAFFE16BE151070824E3CC
:10107E00E351EF16120EE926E351EF1693EC03F04F
:10108E00E451EF1293EC03F0120EE95EE451EF140B
:10109E00006E0CE0E1C201F0010E006E015004E0A2
:1010AE0000360090FF0FFBD70050E21352EC04F015
:0E10BE0052EC04F0E12BD9D7E2C200F0120090
:1010CC00826A0F013A6BFF0E946E948E949C828010
:1010DC009492949094948B828B948B903F0E806E10
:1010EC00386B1F0E926E928692988998546BFF0EF5
:0C10FC00816E830E936E396B606A1200E7
:101108000201E16BDEC2E9FFDFC2EAFFEECFE0F2E7
:10111800E051000A0FE0E0C2E8F298EC03F00201A7
:10112800E12BE151DE25E96E000EDF21EA6EEECFFC
:06113800E0F2EED7120008
:10113E00DEC200F00032009E0032009E0032009EA1
:10114E000032009EE50E0024F66E210EF76E000EA4
:10115E00F722000EF86E000EF8220900F5CF00F00F
:10116E00DFC2E1FFE0C2E2FF00C0E6FF010E0201B6
:10117E00DF25E16E000EE021E26E0F0EDE15006E31
:10118E00E50E0024F66E210EF76E000EF722000E0D
:10119E00F86E000EF8220900F5CF00F000C0E6FF51
:1011AE00020EDF25E16E000EE021E26EE66A12000D
:1011BE0014EC11F09B6A700ED36E9B9CD26A7FDF8B
:1011CE008B82150E0B6E4B0E0C6EBE0E0D6E0D2E13
:1011DE00FED70C2EFCD70B2EFAD70000640E3B6EFA
:1011EE00000E3C6E89980101366B376B000E375D31
:1011FE0002E1800E365D0AE2780E3625E16E010EB2
:10120E003721E26EE66A364B372BF0D7780E0001A7
:10121E00816F010E826FB886B06ACF0EAF6EAC844E
:10122E0050DC030E0B6E080E0C6E770E0D6E0D2E2F
:10123E00FED70C2EFCD70B2EFAD70C0EE86F98ECBF
:10124E0003F0030E0B6E080E0C6E770E0D6E0D2E48
:10125E00FED70C2EFCD70B2EFAD770DD6FDDBF0E2E
:10126E000201DE6F210EDF6F000EE06F99DC0101CF
:10127E00366B376B000E375D02E10A0E365D1BE2F0
:10128E00030E006E000E016E36C104F037C105F07C
:10129E0082EC04F0190E0024E96E000E0120EA6EB5
:1012AE00EECFDEF2EECFDFF2EECFE0F279DC01012F
:1012BE00364B372BDFD7030E0B6E080E0C6E770EE8
:1012CE000D6E0D2EFED70C2EFCD70B2EFAD736DD5B
:1012DE002C0E0201DE6F210EDF6F000EE06F60DC60
:1012EE0052DC0001836B846B800E0201DE6F0F0EE9
:1012FE00DF6FE06B2CEC05F057EC05F0800EDE6F27
:10130E000F0EDF6FE06B330EE16F07DC57EC05F06D
:10131E00800EDE6F0F0EDF6FE06B92DE00C0C9F045
:10132E0057EC05F0F50EDE6F210EDF6F000EE06F4D
:10133E0037DC0001CA6BC9C0DEF2CA0E0201DF6FD4
:10134E00000EE06FF5DECA0EDE6F000EDF6FD5DE2B
:10135E00130EDE6F220EDF6F000EE06F21DC010137
:10136E00366B376B000E375D02E1060E365D2FE2EF
:10137E00800E0201DE6F0F0EDF6FE06B61DE00C0CC
:10138E00C9F0340E0C6EF10E0D6E0D2EFED70C2E16
:10139E00FCD7000000002E0E01013625E16E010E75
:1013AE003721E26EC9C0E6FF0001CA6BC9C0DEF28A
:1013BE00CA0E0201DF6F000EE06FBADECA0EDE6FDC
:1013CE00000EDF6F9ADE0101364B372BCBD71B0E8B
:1013DE000201DE6F220EDF6F000EE06FD7EC05F01C
:1013EE00800E0201DE6F0F0EDF6FE06B29DE00C094
:1013FE00C9F00001CA6BC9C0DEF2CA0E0201DF6F6E
:10140E00000EE06F95DECA0EDE6F000EDF6F75DE2A
:10141E0095DCE30E0201DE6F200EDF6F000EE06F33
:10142E00D7EC05F0D08E9F8A9E8AAB88F28CF28E16
:10143E000001856B866B570E0201DE6F200EDF6F8B
:10144E00000EE06FD7EC05F0EBDD140E0201DE6F3F
:10145E00000EDF6F7CDD240EAD6E70DC000E3E18CC
:10146E0002E1000E3D1801E1F9D7230EAD6E66DCE8
:10147E000001856B866B0101366B376B000E375D95
:10148E0002E1100E365D17E236C100F037C101F0F1
:10149E00003600900136003600900136F80E00241A
:1014AE00E16E010E0120E26EE66AE66AE66AE66A1F
:1014BE00364B372BE3D7366B376B000E375D02E1B9
:1014CE00400E365D0AE2410E3625E16E000E3721E2
:1014DE00E26EE66A364B372BF0D78B82DAEC04F0ED
:1014EE00AC0EDE6F210EDF6F000EE06FD7EC05F055
:1014FE00A8EC03F023DCB80E0201DE6F200EDF6FC6
:10150E00000EE06FD7EC05F00001CA6BCA0E0201A7
:10151E00DE6F000EDF6F230EE06F220EE16F000E06
:10152E00E26F55DDCA0E0201DE6F000EDF6FF9ECC1
:10153E0005F0150E0B6E4B0E0C6EBE0E0D6E0D2EB7
:10154E00FED70C2EFCD70B2EFAD70000050E3B6EE5
:10155E00000E3C6E780E0001876F010E886FF29EB2
:10156E00800E0201DE6F0F0EDF6FE06B2CEC05F0CC
:10157E00800EDE6F0F0EDF6FE06BCC0EE16F94EC22
:10158E0005F0800EDE6F0F0EDF6FE06B440EE16F25
:10159E0094EC05F0040E0C6EE40E0D6E0D2EFED7BF
:1015AE000C2EFCD70000800EDE6F0F0EDF6FE06B8F
:1015BE002CEC05F0800EDE6F0F0EDF6FE06BCC0EA5
:1015CE00E16F94EC05F0800EDE6F0F0EDF6FE06BB7
:1015DE00BE0EE16F94EC05F0800EDE6F0F0EDF6F26
:1015EE00E06B2EDD00C0DAF2000EDB6F800EDE6FD8
:1015FE000F0EDF6FE06B24DD00C003F0026ADA51DC
:10160E000224006EDB510320016E00C0DCF201C02B
:10161E00DDF200C0DEF201C0DFF2CA0EE06F020E94
:10162E00E16FAEEC06F0780E0001876F010E886F49
:10163E0081C0DEF282C0DFF2730E0201E06F210E76
:10164E00E16F000EE26FC3DC81C0DEF282C0DFF21A
:10165E00CA0E0201E06F020EE16FAAEC04F081C027
:10166E00DEF282C0DFF249DDA5EC06F00101366B39
:10167E00376B000E375D02E1200E365D0AE2410E39
:10168E003625E16E000E3721E26EE66A364B372BB9
:10169E00F0D787C0DEF288C0DFF269DC280EDE6F7D
:1016AE00000EDF6F54DC81C0DEF282C0DFF225DD7A
:1016BE00A5EC06F0F28E000E3E1802E1000E3D186B
:0A16CE0001E1F9D789784BD7FFD767
:1022280010EE19F0240E006E010E016E080EF66E07
:0E223800210EF76E000EF86E60EC05F012003D
:1016D80000000000000000001010101010001000A2
:1016E800242424000000000024247E247E242400D6
:1016F800183E403C027C1800006264081026460030
:10170800304830568888760010102000000000000D
:101718001020404040201000201008080810200029
:10172800004438FE384400000010107C10100000FF
:1017380000000000001010200000007E00000000E3
:1017480000000000001010000002040810204000F3
:101758003C42464A52623C001030501010107C0047
:101768003C42020C30427E003C42021C02423C00D9
:1017780008182848FE081C007E407C0202423C00F3
:101788001C20407C42423C007E420408101010009D
:101798003C42423C42423C003C42423E0204380049
:1017A8000010100000101000001010000010102091
:1017B800081020402010080000007E00007E000075
:1017C80010080402040810003C4202040800080043
:1017D8003C425E525E403C00182442427E42420037
:1017E8007C22223C22227C001C22404040221C00F9
:1017F80078242222222478007E22283828227E007B
:101808007E222838282070001C2240404E221E00CC
:101818004242427E424242003810101010103800F6
:101828000E04040444443800622428302824630049
:101838007020202020227E0063554941414141000B
:1018480062524A46424242003C42424242423C00C4
:101858007C22223C202070003C4242424A3C030049
:101868007C22223C282472003C42403C02423C003C
:101878007F49080808081C004242424242423C0094
:10188800414141412214080041414149494936003A
:1018980041221408142241004122140808081C009F
:1018A8007F42040810217F00784040404040780083
:1018B800804020100804020078080808080878000A
:1018C800102844820000000000000000000000FF13
:1018D800101008000000000000003C023E423F00DB
:1018E8006020202E31312E0000003C4240423C0056
:1018F8000602023A46463B0000003C427E403C005D
:101908000C1210381010380000003D42423E027C94
:1019180060202C3222226200100030101010380093
:10192800020006020242423C602024283028260099
:10193800301010101010380000007649494949004D
:1019480000005C624242420000003C4242423C00CD
:1019580000006C32322C20700000364C4C34040EDF
:1019680000006C322220700000003E403C027C00E7
:1019780010107C1010120C000000424242463A003F
:10198800000041412214080000004149494936003D
:10199800000044281028440000004242423E027CD5
:1019A80000007C0810207C000C10106010100C0047
:1019B8001010100010101000300808060808300039
:1019C800324C0000000000001C14141C0000000031
:1019D8003C4240423C0C023C0044004444443E002B
:1019E8000C003C427E403C003C4238043C443E00F3
:1019F800420038043C443E00300038043C443E0079
:101A08003C2424243C00000000003C40403C061CD0
:101A18003C423C427E403C0042003C427E403C000E
:101A280030003C427E403C002400180808081C0096
:101A38007C823010101038003000180808081C008C
:101A4800421824427E4242001818003C427E42005E
:101A58000C007C2038207C000000330C3F443B0005
:101A68001F24447F444447001824003C42423C0061
:101A78000042003C42423C002010003C42423C00F4
:101A88001824004242423C002010004242423C00DE
:101A980000420042423E023C4218244242241800BE
:101AA8004200424242423C0008083E40403E08088C
:101AB8001824207020427C0044287C107C101000E0
:101AC800F84C78444F4445E61C12107C1010906086
:101AD8000C0038043C443E000C00180808081C00A0
:101AE8000408003C42423C000004084242423C00D8
:101AF800324C007C42424200324C0062524A46005C
:101B08003C44443E007E000038444438007C0000D9
:101B18001000102040423C000000007E40400000C1
:101B28000000007E0202000042C448F629438C1FD0
:101B380042C44AF62A5F82020010001010101000FA
:101B480000122448241200000048241224480000EF
:101B5800228822882288228855AA55AA55AA55AAD9
:101B6800DB77DBEEDB77DBEE1010101010101010B7
:101B780010101010F01010101010F010F0101010BD
:101B880014141414F414141400000000FC14141495
:101B98000000F010F01010101414F404F4141414CD
:101BA80014141414141414140000FC04F41414145D
:101BB8001414F404FC00000014141414FC000000B5
:101BC8001010F010F000000000000000F0101010DD
:101BD800101010101F00000010101010FF0000005F
:101BE80000000000FF101010101010101F1010102F
:101BF80000000000FF00000010101010FF1010106F
:101C080010101F101F10101014141414171414148B
:101C1800141417101F00000000001F1017141414CC
:101C28001414F700FF0000000000FF00F71414145C
:101C380014141710171414140000FF00FF000000FC
:101C48001414F700F71414141010FF00FF0000001C
:101C580014141414FF0000000000FF00FF101010FF
:101C680000000000FF141414141414141F000000C2
:101C780010101F101F00000000001F101F10101070
:101C8800000000001F14141414141414FF14141466
:101C98001010FF10FF10101010101010F0000000AE
:101CA800000000001F101010FFFFFFFFFFFFFFFFE5
:101CB80000000000FFFFFFFFF0F0F0F0F0F0F0F0A0
:101CC8000F0F0F0F0F0F0F0FFFFFFFFF0000000098
:101CD8000000314A444A3100003C427C427C40408A
:101CE800007E424040404000003F54141414140049
:101CF8007E42201820427E0000003E4848483000BE
:101D0800004444447A40408000334C0808080800E6
:101D18007C1038444438107C1824427E4224180031
:101D280018244242242466001C20183C42423C00ED
:101D3800006295899562000002043C4A523C40804A
:101D48000C10203C20100C003C424242424242000F
:101D5800007E007E007E000010107C1010007C00C9
:101D68001008040810007E000810201008007E00EB
:101D78000C1212101010101010101010109090600B
:101D88001818007E0018180000324C00324C000071
:101D9800304848300000000000000018180000001B
:101DA80000000000180000000F08080808C82818DC
:101DB8007844444444000000304810207800000073
:101DC80000003C3C3C3C000000000000000000001B
:101DD80000000000000000000000000000000000FB
:101DE80000000000000000000000000000000000EB
:101DF80000000000000000000000000000000000DB
:101E080000000000000000000000000000000000CA
:101E180000000000000000000000000000000000BA
:101E280000000000000000000000000000000000AA
:101E3800000000000000000000000000000000009A
:101E4800000000000000000000000000000000008A
:101E5800000000000000000000000000000000007A
:101E6800000000000000000000000000000000006A
:101E7800000000000000000000000000000000005A
:101E8800000000000000000000000000000000004A
:101E9800000000000000000000000000000000003A
:101EA800000000000000000000000000000000002A
:101EB800000000000000000000000000000000001A
:101EC800000000000000000000000000000000000A
:101ED800204469726563746F7279203A20433A5CD2
:101EE8005F4D696B726F435C5F4D657350726F6ACB
:101EF8006574735F4D696B726F435C5F313846324E
:101F0800364B32325F424153455F546573745F31DB
:101F1800325F4D617472696365733878385F486FF2
:101F280072697A6F6E74616C65735F313931302014
:031F38000D0A008F
:101F3B0020536F75726365203A20426173655F3180
:101F4B00384632364B32325F746573745F64656644
:101F5B00696C656D656E745F315F626C6F635F6436
:101F6B00655F345F4D6174726963653878385F48BB
:101F7B005F2056657273696F6E203A2032303230B3
:091F8B005F30365F30380D0A00AA
:101F94002050726F6A6574203A20426173655F3124
:101FA400384632364B32325F746573745F646566EB
:101FB400696C656D656E745F345F4D6174726963DD
:101FC400653878385F485F323032305F30362E6D96
:071FD400637070690D0A0043
:101FDB0020535049206269742062616E67203A2059
:101FEB000D0A205243303D434C4F434B202052436C
:101FFB00313D4353205243323D44494E202D2D2D2C
:0E200B003E204D41583732313920200D0A0059
:10201900205465726D696E616C207574696C6973A1
:10202900E920636F6D6D6520706F696E7420642798
:102039006172726574206465726F756C656D656E29
:0E204900742070726F6772616D6D650D0A0014
:10205700205465737420696E74657272757074208C
:1020670054696D657231202032302078203130304C
:10207700206D73656320736F697420327365632005
:032087000D0A003F
:10208A00204D6F64756C652064652034204D617441
:10209A007269636520482038783820617665632044
:0E20AA004D41583731323920434D530D0A0055
:1020B80020416666696368652054657874204649DE
:1020C800584520656E204173636369202866726FE6
:0B20D8006D204352616D31290D0A009C
:1020E30020496E697420496E74657272757074202C
:1020F30054696D6572312020262055415254205277
:0521030058200D0A0048
:10210800502100D81E00941F003B1F008A20001990
:0E2118002000D22100DB1F00052200952100CF
:0421260000000000B5
:02212A0014009F
:10212C00205465737420536F6E64652041204F57A3
:10213C00532044533138423230207375722052434D
:04214C00300D0A0048
:10215000204D696B726F6320372E362E30200D0AAA
:10216000204D4355203A2031384632364B3232200A
:032170000D0A0055
:10217300205061756C666A756A6F40667265652E7C
:1021830066722054656D702E2044533138423230CC
:022193003D000D
:10219500204F5753204453313842323020737572E3
:0721A500205241310D0A0038
:1021AC00436C6561722034204D61747269636520E3
:0321BC000D0A0009
:1021BF002050726573656E746174696F6E203A207A
:0321CF000D0A00F6
:1021D20020416C696D203D332E365620E020355665
:0321E2000D0A00E3
:1021E5003031323334353637383941424344454648
:1021F5002046616D696C7920436F6465203A200043
:0E22050020464F53433D2031362E300D0A0047
:0822130020494431203D200068
:08221B0020204352433D200046
:052223003031323300F0
:020000040030CA
:0D00010038193CFFBF81FF0FC00FE00F401A
:00000001FF
